:1000000012C02AC029C028C027C026C025C024C0CD
:1000100023C022C021C020C01FC01EC01DC01CC0E4
:100020001BC01AC019C011241FBECFEDCDBF10E0F8
:10003000A0E6B0E0E2E9F5E002C005900D92A0363E
:10004000B107D9F710E0A0E6B0E001C01D92AC36D0
:10005000B107E1F702D09BC2D3CF8FE881BB87EF16
:1000600087BBC29A84E090E078D28093650083E0F9
:1000700090E073D28093640082E090E06ED280932F
:10008000680081E090E069D28093630080E090E0B6
:1000900064D280936900D4E001E010E0CC24DD2438
:1000A000FF24F394C0E00F2EF3E0EF2EF02D40D1AB
:1000B00080936A008B3009F0D8BB3AD180936200FC
:1000C00037D18093660034D18093670031D180931B
:1000D0006B00A80120916700909163002913A6018D
:1000E000980160916600909168006913960142231F
:1000F00053232F2D30916A009091650039132C2FD6
:100100009F2D609162003091640063139C2F29231E
:1001100030E042235323980190916900891396019E
:10012000242335232115310521F1C39AB39915C034
:100130008FE19EE40197F1F700C00000B3990DC074
:1001400083E088BB2FEF31E14AE721503040404047
:10015000E1F700C0000018BA80DFE8BAC0936A0077
:10016000C0936200C0936600C0936700C0936B00A9
:100170009ECF8E2DD8BB2FEF31EE44E02150304082
:100180004040E1F700C0000018BA2FEF31EE44E024
:10019000215030404040E1F700C00000D8BBC09380
:1001A0006A00C0936200C0936600C0936700C0936A
:1001B0006B008150F9F67BCFCF93DF9382E088BB51
:1001C0002FEF31EE44E0215030404040E1F700C0D5
:1001D000000084E088BB849BFECFAAD080936A0095
:1001E000A7D080936200A4D080936600A1D08093B2
:1001F00067009ED080936B0021E030E04091670063
:1002000090916300491711F020E030E041E050E0A8
:100210006091660090916800691711F040E050E02D
:100220004223532361E020916A00909165002913D5
:1002300060E091E03091620020916400321390E020
:10024000692370E04623572321E030E09091690054
:10025000891711F020E030E02423352321153105E2
:1002600009F44AC0D2E0D8BB8FEF91EEA4E08150F0
:100270009040A040E1F700C00000C4E0C8BB2FEFF1
:1002800031EE44E0215030404040E1F700C0000032
:100290004FD0809365004CD08093640049D0809308
:1002A000680046D08093630043D08093690084E067
:1002B00090E06091650059D183E090E06091640026
:1002C00054D182E090E0609168004FD181E090E0ED
:1002D000609163004AD180E090E06091690045D16F
:1002E000D8BB8FEF91EEA4E081509040A040E1F7A1
:1002F00000C00000C8BBB1DE83E094E098BB2FEFE4
:1003000031EE44E0215030404040E1F700C00000B1
:1003100018BA2FEF31EE44E0215030404040E1F771
:1003200000C0000098BB815049F7DF91CF9108953C
:100330007F928F929F92AF92BF92CF92DF92EF9275
:10034000FF920F931F93CF93DF93109261000F2EB4
:10035000FEEFFF2EF02DC1E0EE246894E1F80F2EA1
:10036000F3E0DF2EF02D0DEFCC246894C2F80F2EB1
:10037000F5E0BF2EF02D0F2EF6E0AF2EF02D1BEF87
:100380000F2EF7E09F2EF02D8824689483F80F2E0F
:10039000F9E07F2EF02DD7EFCAC0F2BA8FE097E2D6
:1003A0000197F1F700C0000084990EC0AFE1BEE4F0
:1003B0001197F1F700C00000849906C0C093600057
:1003C000C0936100849BFECF85990EC08FE19EE4AF
:1003D0000197F1F700C00000859906C0E092600027
:1003E000C0936100859BFECF86990EC0AFE1BEE44D
:1003F0001197F1F700C00000869906C0D092600006
:10040000C0936100869BFECF02BB8FE097E201970D
:10041000F1F700C0000084990EC0AFE1BEE411976F
:10042000F1F700C00000849906C0C0926000C0933C
:100430006100849BFECF85990EC08FE19EE40197F9
:10044000F1F700C00000859906C0B0926000C0932B
:100450006100859BFECF86990EC0AFE1BEE4119787
:10046000F1F700C00000869906C0A0926000C0931A
:100470006100869BFECF12BB8FE097E20197F1F7F8
:1004800000C0000084990EC0AFE1BEE41197F1F7FF
:1004900000C00000849906C090926000C093610083
:1004A000849BFECF85990EC08FE19EE40197F1F702
:1004B00000C00000859906C080926000C093610072
:1004C000859BFECF86990EC0AFE1BEE41197F1F790
:1004D00000C00000869906C070926000C093610061
:1004E000869BFECFD2BB8FE097E20197F1F700C069
:1004F000000085990FC0AFE1BEE41197F1F700C08D
:100500000000859907C08AE080936000C093610075
:10051000859BFECF84990BC08FEF9DE3A9E48150AA
:100520009040A040E1F700C00000849B45DE809130
:100530006100813009F031CF8091600090E0DF915F
:10054000CF911F910F91FF90EF90DF90CF90BF90D0
:10055000AF909F908F907F900895E199FECF1FBA42
:100560008EBBE09A99278DB30895262FE199FECF8F
:100570001FBA8EBBE09A81500DB2021639F01CBA38
:100580002DBB0FB6F894E29AE19A0FBE0895F89445
:02059000FFCF9B
:00000001FF
